:020000020000FC
:020000000CC131
:0200080036C000
:10000E007DC096C00905060A0901050406020A0804
:10001E00DD24EE1841E1001F111F4A9509F40895E1
:10002E00DD1CEE1CD21AE30A20F4D20EE31E8894D5
:10003E00F2CF0894F0CF5527442760E136952795E7
:10004E0010F4400F511F57954795379527956A9590
:10005E00B9F70895662019F4772009F42AC0F0E064
:10006E00E1E06E1A7F0A25C0EF93FF930F930FB74F
:10007E0085FDF0CF81FF31C0AA95F0E0E1E06E0E74
:10008E007F1E64147504A8F06624772482FF1EC0B8
:10009E00BE0ECF1EB395B81508F0BB27E1E0F0E019
:1000AE009E1AAF0A31F48D7FE4E17E2E66248062C3
:1000BE00AA270F92EEE0E80DFF27EB0FC89508BABE
:1000CE000F900FBF0F91FF91EF911895BE1ACF0AA7
:1000DE00BA9512F4B82DBA95E1CFAA2311F0AA95CC
:1000EE00F0CF84FD05C0FF27E8E9A0818061E1CF54
:1000FE00FF27F8BBE7E9A0818F7EE3CFFF93EF9355
:10010E000F930FB70F930CB15C990CC0FF27E32D23
:10011E0001930D3019F48160E0E603C0E43709F471
:10012E00E0E63E2E0F910FBF0F91EF91FF911895C4
:10013E000F930FB70F93121429F455980F910FBF09
:10014E000F911895EF93FF93FF27E22D0191EC3756
:10015E0009F4E0E62E2E0CB9FF91EF91EFCF10E2ED
:10016E0000270A95F1F71A95E1F70895F8941214FD
:10017E00FF27E12D0193EC3709F4E0E61E2E559A88
:10018E0078940895C8953196002039F0002DFF938C
:10019E00EF93ECDFEF91FF91F5CF0895FF270191DB
:1001AE00EF93E4DFEF91FF270D3009F0F8CF0895BC
:1001BE0074E0EAE3F7E0972F8894991FE90F08F4AB
:1001CE00F395C895202DE395C895302D21DF005D60
:1001DE00CDDF0D2D1E2D7A9562F70DE0C7DF089548
:1001EE00C72FDD270881003211F4C395FBCF7C2F7A
:1001FE000895C72FDD27C895002011F47C2F089590
:10020E0031960991001509F4F6CF08950FED0DBF43
:10021E0000E6102E202E04E0802E00E6302E8827D9
:10022E000FE007BB002708BB08E90AB900E409B9CB
:10023E00BB24CC24BB27DD27CAE808EE099303E0D4
:10024E000993C8E808EE099303E00993C4E902E3B1
:10025E00088301E0C8E90883C7E9088347D104E6AB
:10026E00402E552466247724AA2700270FBD09E0C7
:10027E000EBD00270BBD0AE90ABD00E409BF81FFD0
:10028E0001C063C0789480FFFECFF894FF27E0E6AC
:10029E00DD27C4E7019109930D30E1F778948E7F45
:1002AE0074E79EDFE4EBF6E0A4DF11F4F2D0E7CFC3
:1002BE0081FD3CC0E6ECF6E09CDF11F459D1DFCFB6
:1002CE00EAECF6E096DF11F459D1D9CFE2EDF6E083
:1002DE0090DF11F498D1D3CFEAEDF6E08ADF11F476
:1002EE00A8D1CDCFE6EBF6E084DF11F438D1C7CF3D
:1002FE00E0ECF6E07EDF11F445D1C1CFE2EEF6E0A0
:10030E0078DF11F448D1BBCFEAEEF6E072DF11F4DC
:10031E004CD1B5CFE2EFF6E06CDF11F44FD1AFCF99
:10032E00EAEFF6E066DF11F452D1A9CFE4E1F7E08F
:10033E0029DFA5CFF894062D172D78940023D1F739
:10034E001123C1F7F8948F7D089504E1702E662471
:10035E0080627894EFDFAFE383FD3BC0FF27FDBDE6
:10036E00F395FCBDDD27CEE849905880789483FF45
:10037E001CC080FF0FC08E7FDD27C0E608810236CD
:10038E0049F4DD27C2E9F8949990A880992009F4E0
:10039E0093944FC0DD27C2E909911881F89409158D
:1003AE001A0508F046C078940DC080FF0BC08E7FF2
:1003BE00DD27C0E60881023629F4F89401E0902E7C
:1003CE00AA24789481FDD3CFE0E1F7E0DBDEB2DF43
:1003DE0056CFFF27E2E99192A082662751E039D0ED
:1003EE00FDBDF395FCBDF8944C2E5D2E78945F5FA9
:1003FE006F4F2FD0FF27EEE8019110814016510666
:10040E0010F009F009C0E2E90191108109191A09E9
:10041E00E2E901931083A6CFE0E90191108109155D
:10042E001A0538F481FFD0CFA03408F4FBCFAFE328
:10043E00DACF78945E5F6F4F25D0F894AFE3F894DF
:10044E004C2E5D2E78941ED081FFBECFA034E0F3EB
:10045E00F5CF052F162F91E08894179507959A954D
:10046E00D9F7202F312FECE801911081D1DDC02F6B
:10047E00D12FE5E9019110810C171D0710F4C02F43
:10048E00D12F08955150604010F460E051E0E1DF4B
:10049E000895ECE1F7E076DE0895972FC72FDD275C
:1004AE000991003318F00A3308F4FACF21977C2F04
:1004BE00791BD1F07630C0F47C2FEAE3F7E0EE241E
:1004CE00DD2411270A910053C8953196202DC89529
:1004DE003196302DB0DDD20EE31E30F0C91791F7F4
:1004EE00442311F48894089508940895DD27CAE8EA
:1004FE000991188192E08894001F111F9A95D9F7DF
:10050E00C8E82991388184DD29E63FE391E088949B
:10051E00379527959A95D9F78EDD442311F00FEF75
:10052E001FEFCCE82993388307EA1DEFC8E829911D
:10053E0038816EDDCEE80993188307EA1DEFC4E912
:10054E002881332765DDC5E9099318830895E4E111
:10055E00F7E018DE0895E0E1F7E014DE089540DEDE
:10056E009CDFA8F3DD27CAE8D992E992BFDFF3CF6B
:10057E0037DE93DF60F3BD2CCE2CEDCF0B2D1C2D73
:10058E0017DE08952DDE89DF10F3DD27C8E8D99236
:10059E00E992ACDFE0CF24DE80DFC8F2EE20B9F6C0
:1005AE00DD27C4E9D882A2DFD6CF1ADE76DF78F255
:1005BE00EE2069F6DD27C8E9D882CDCF11DE6DDFDA
:1005CE0030F2EE2021F6DD27C7E9D882C4CF08DE4F
:1005DE0064DF68F1EE2059F502E0D01640F5DD201B
:1005EE0049F008E0801621F1F894802E8894BB1F04
:1005FE007894B1CF04E08016D9F0F894802E8894C8
:10060E00B7957894A8CFECDDC72FDD2708810D3282
:10061E0011F0846002C073958B7F3FDF40F000279E
:10062E00D016E00629F09D2CAE2C17D008958FCF52
:10063E0092CFD6DD32DFD8F3DB14EC04C9F338F0F9
:10064E008460DB18EC089D2CAE2C07D008958B7FB0
:10065E009B2CAC2C9D18AE08F8CF90E09916A906ED
:10066E0009F40895CCE8DD270991188109171907B7
:10067E0009F0886066247724092D1A2D8894179521
:10068E000795C0E909931883F89482600895E4E011
:10069E00F7E0DD27C0E6C895319609920020D9F71C
:0406AE0081600895CA
:1006B4003F0072616D7074696D65000066726571EA
:1006C40000007365740073746174757300006D6F5A
:1006D400766572656C006D6F7665616273006D6935
:1006E4006E6672657100647574796F6E000064756E
:1006F40074796F66660068616C6673746570000077
:1007040068616C667374657020300D006F6B0D004A
:100714006572726F720D0000446F75626C65466F8E
:10072400782053746570706572205265762E20317E
:100734002E30630D000001000A006400E803102756
:00000001FF
